:020000040800F2
:10000000680B0024AD020008E5150008E3150008A0
:10001000B9020008C1030008B11E0008000000007A
:10002000000000000000000000000000E9150008CA
:100030004D04000800000000E715000899160008AC
:10004000C7020008C7020008C7020008C70200086C
:10005000C7020008C7020008C7020008C70200085C
:10006000C7020008C7020008C7020008C70200084C
:10007000C7020008C7020008C7020008C70200083C
:10008000C7020008C7020008C7020008C70200082C
:10009000C7020008C7020008C7020008C70200081C
:1000A000C7020008C7020008C7020008C70200080C
:1000B000C7020008C7020008C7020008C7020008FC
:1000C000C7020008C7020008C7020008C7020008EC
:1000D000C70200086D1E0008C7020008C70200081A
:1000E000C7020008C702000800000000C70200089D
:1000F000C7020008C7020008C7020008C7020008BC
:10010000C7020008C7020008C7020008C7020008AB
:10011000C7020008C7020008C7020008C70200089B
:10012000C7020008C7020008C7020008C70200088B
:10013000C7020008C7020008C7020008C70200087B
:1001400000000000000000000000000000000000AF
:10015000C7020008C7020008C7020008C70200085B
:10016000C7020008C7020008C7020008C70200084B
:10017000C7020008C7020008C7020008C70200083B
:10018000C7020008C7020008C7020008C70200082B
:10019000C7020008C7020008C7020008C70200081B
:1001A000C7020008C7020008C7020008C70200080B
:1001B000C7020008C7020008C7020008C7020008FB
:1001C000C7020008C7020008C7020008C7020008EB
:1001D000C7020008C7020008C7020008C7020008DB
:1001E000C7020008C7020008C7020008C7020008CB
:1001F000C7020008C7020008C7020008C7020008BB
:10020000C7020008C7020008C7020008C7020008AA
:10021000C7020008C7020008C7020008C70200089A
:10022000C7020008C7020008C7020008000000005B
:10023000C7020008C702000800000000C70200084B
:10024000C7020008C7020008C7020008C70200086A
:10025000C7020008C7020008C7020008C70200085A
:10026000C7020008C7020008C7020008C70200084A
:10027000C7020008C7020008C7020008000000000B
:10028000C702000800000000C702000800000000CC
:1002900000000000C7020008DFF80CD000F07EF874
:1002A00000480047E1200008680B0024064880470A
:1002B00006480047FEE7FEE7FEE7FEE7FEE7FEE74B
:1002C000FEE7FEE7FEE7FEE79D160008990200083C
:1002D0002DE9F05F0546002092469B46884606467B
:1002E000814640241BE0284641464746224600F00E
:1002F00045F853465A46C01A914110D31146184644
:10030000224600F02CF82D1A67EB01084F462246D2
:100310000120002100F023F817EB00094E41201EB8
:10032000A4F10104DFDC484631462A464346BDE8D5
:10033000F09F30B50B46014600202022012409E041
:1003400021FA02F59D4205D303FA02F5491B04FA8E
:1003500002F52844151EA2F10102F1DC30BD202A6D
:1003600004DB203A00FA02F1002070479140C2F10C
:10037000200320FA03F3194390407047202A04DB3E
:10038000203A21FA02F00021704721FA02F3D0400E
:10039000C2F120029140084319467047064C074DB0
:1003A00006E0E06840F0010394E807009847103445
:1003B000AC42F6D3FFF774FF9C210008BC21000873
:1003C000FEE70000F0B5BFF34F8FBFF36F8F1D49FD
:1003D00000200860BFF34F8FBFF36F8F1A4C216866
:1003E00041F400312160BFF34F8FBFF36F8F164987
:1003F00070310860BFF34F8F081F006843F6FF7528
:10040000104E1036C0F34E31C0F3C90305EA411255
:10041000184642EA80773760401EFAD2491EF5D26C
:10042000BFF34F8F206840F480302060BFF34F8FC0
:10043000BFF36F8F03484C30016841F00401016045
:10044000F0BD000050EF00E014ED00E07047000048
:1004500010B528B190F83510022903D080214165EC
:10046000012010BD1D4A4FF4956301688C189C4211
:1004700007D8042280F83520086820F001000860C1
:1004800029E00C6824F00E040C6001680A440A6834
:1004900022F001020A60016E0A6822F480720A608A
:1004A00090F85C30012202FA03F10D4B1960D0E99B
:1004B00019134B60C16E31B10B6823F480730B606C
:1004C000D0E91C134B60002180F8341080F83520EF
:1004D000016D01B18847002010BD0000F0FFFDBF95
:1004E000045402580248016841F00101016070475C
:1004F000200400582DE9F84F6C4C00224FF0B04A10
:100500004FF0010B4FF0030E4FF00F090B680BFA81
:1005100002F73B40BB4270D14D68022D01D0122D35
:1005200012D1D50800EB850CDCF820605507ED0EE4
:1005300009FA05F826EA0806D1F8108008FA05F845
:1005400048EA0608CCF82080D0F80080560091F8E0
:1005500004C00EFA06F50CF0030C28EA05080CFAA4
:1005600006FC4CEA080CC0F800C0D1F804C0BCF18D
:10057000010F08D0BCF1020F05D0BCF1110F02D061
:10058000BCF1120F16D1D0F808C0D1F80C802CEABB
:10059000050C08FA06F848EA0C08C0F80880D0F8FC
:1005A00004C02CEA070C0F79C7F30017974047EAFD
:1005B0000C074760C768AF438D68B5403D43C560D1
:1005C0004D68ED006BD53A4D2E6846F002062E6060
:1005D0002D6822F0030606F1B04605F002050095ED
:1005E000D6F808C495072F0F09FA07F52CEA050C71
:1005F000304DA84202D100252EE050E02E4DA842F9
:1006000001D1012528E02D4DA84201D1022523E08A
:100610002B4DA84201D103251EE02A4DA84201D14D
:10062000042519E0284DA84201D1052514E0274DE5
:10063000A84201D106250FE0254DA84201D107258A
:100640000AE0244DA84201D1082505E0224DA84228
:1006500001D1092500E00A25BD4045EA0C05C6F890
:10066000085425684E689D43F60300D51D43256058
:1006700065684E689D43B60300D51D436560DAF892
:10068000005056464F689D43FF0200D51D4335601C
:1006900075684F689D43BF0200D51D437560521CAD
:1006A000102AFFF433AFBDE8F88F00008000005837
:1006B000F44402580000025800040258000802588E
:1006C000000C02580010025800140258001802587A
:1006D000001C02580020025800240258014880687B
:1006E0007047000014000024024881680278114419
:1006F0008160704714000024032010B500F058F802
:100700000F2000F007F808B1012010BD00F022F81A
:10071000002010BD70B50D4D04464FF47A71287855
:10072000B1FBF0F00A490968B1FBF0F000F086FD7A
:1007300048B9102C07D200222146501E00F018F8AC
:1007400000206C6070BD012070BD0000140000240A
:10075000000000247047002809DB012100F01F027F
:1007600091404009800000F1E020C0F8001170477E
:100770000E4BF0B41B68C3F30223C3F10704042C2F
:1007800000D904241D1D072D01D2002300E0DB1E2B
:10079000012606FA04F56D1E0D409D409E40761E12
:1007A000164045EA0601F0BC01F094BB0CED00E0F8
:1007B000064A00F0070110684FF6FF03184040EAB0
:1007C0000120034908431060704700000CED00E071
:1007D0000000FA0510B500F05BFA084909684FF40B
:1007E000807292FAA2F201F47061B2FA82F2D14000
:1007F000034A515CC8400349086010BD18440258C0
:10080000742100080000002410B500F0FBF907492E
:100810000968102292FAA2F201F07001B2FA82F293
:10082000D140034A515CC84010BD0000204402582A
:1008300074210008364930B50A68096812F00302CD
:10084000344BC1F305311B68334C03F010032468AB
:10085000DFED320AB7EE001AC4F3CC0414FB03F345
:1008600000EE103A2E4BB8EE400A07D02D4C012A6C
:1008700001D0022A4AD0B4FBF1F10BE0244C283C11
:1008800022689506284A03D52468C4F3C104E240CF
:10089000B2FBF1F101EE901A1968B8EE612AC1F3CA
:1008A000080101EE901A1968F8EE611A40EE201A5C
:1008B00031EE810A22EE000AC1F34621491C00EE06
:1008C000901AF8EE600A80EE201AFCEEC10AC0ED24
:1008D000000A1968C1F30641491C00EE901AF8EEAF
:1008E000600A80EE201AFCEEC10AC0ED010A196808
:1008F000C1F30661491C00EE901AF8EE600A80EE22
:10090000201ABCEEC10A80ED020A30BD074ABFE7DB
:10091000284402582C4402583C4402580000003934
:100920003844025800093D000090D00340787D0112
:10093000364930B50A68096812F00302344BC1F336
:1009400005511B68334C03F480732468DFED320AD1
:10095000B7EE001AC4F3CC0414FB03F300EE103A14
:100960002E4BB8EE400A07D02D4C012A01D0022AA6
:100970004AD0B4FBF1F10BE0244C283C22689506E8
:10098000284A03D52468C4F3C104E240B2FBF1F164
:1009900001EE901A1968B8EE612AC1F3080101EE60
:1009A000901A1968F8EE611A40EE201A31EE810AA9
:1009B00022EE000AC1F34621491C00EE901AF8EE1F
:1009C000600A80EE201AFCEEC10AC0ED000A196828
:1009D000C1F30641491C00EE901AF8EE600A80EE61
:1009E000201AFCEEC10AC0ED010A1968C1F30661C4
:1009F000491C00EE901AF8EE600A80EE201ABCEE58
:100A0000C10A80ED020A30BD074ABFE728440258F8
:100A10002C44025844440258000000394044025813
:100A200000093D000090D00340787D012DE9F0479A
:100A3000DFF8BC9104460E46D9F8000000F007002C
:100A4000B0420CD2D9F8001021F007013143C9F8A7
:100A50000010D9F8000000F00700B0427ED12078E5
:100A6000DFF89081800707D5D8F80010E26821F000
:100A70000F011143C8F800102078C00762D0D8F8E1
:100A80000010A26821F470611143C8F800105949A0
:100A90006068183902281CD003281DD00968012875
:100AA0001DD04907002960DA524F083F396821F00C
:100AB000070101433960FFF711FE0546606841F206
:100AC0008831022813D003281ED001288A4627D057
:100AD00034E009688903E5E709688901E2E7C905A7
:100AE000E0E7FFF7FBFD411B514501D923E08A46B2
:100AF0003868C0F3C2000228F3D123E0FFF7EEFD0F
:100B0000411B514501D916E08A463868C0F3C2003E
:100B10000328F3D116E0FFF7E1FD411B51450AD848
:100B20003868C0F3C2000128F5D10BE0FFF7D6FD0D
:100B3000411B514502D90320BDE8F087386810F009
:100B4000380FF3D1D9F80010484601F00701B1423F
:100B50000DD9016821F00701314300E005E0016093
:100B6000006800F00700B04201D00120E4E72078DF
:100B7000400707D5D8F80010226921F07001114311
:100B8000C8F80010207801071B4805D50168626984
:100B900021F07001114301602178C90605D5016873
:100BA000A26921F4E061114301602078800607D535
:100BB0001149091D0868E26920F0700010430860BF
:100BC00000F066F8D8F800104FF4807292FAA2F2A2
:100BD00001F47061B2FA82F2D140084A515CC84017
:100BE000074908600F20FFF795FD0020A4E70000EB
:100BF00000200052184402581C4402587421000876
:100C00000000002410B5FFF7E5FD0849096801223E
:100C100092FAA2F201F00F01B2FA82F2D140044A34
:100C2000515CC8400349086010BD000018440258D8
:100C3000742100080400002410B5FFF7E3FF074902
:100C40000968102292FAA2F201F07001B2FA82F25F
:100C5000D140034A515CC84010BD00001C440258FA
:100C60007421000810B5FFF7CDFF074909684FF45C
:100C7000807292FAA2F201F4E061B2FA82F2D140FB
:100C8000024A515CC84010BD1C440258742100083F
:100C90003548F0B50068364D10F03801334809D0BA
:100CA0000411082904D0334E10290BD018290BD079
:100CB0002046F0BD29688906FBD52968C1F3C1012A
:100CC000C840F0BD3046F0BD274918310A680968B0
:100CD00012F00302284BC1F305111B68274F03F0E4
:100CE00001033F68DFED260AB7EE001AC7F3CC0711
:100CF00017FB03F300EE103A224BB8EE400A06D081
:100D0000012A01D0022A2BD0B4FBF1F008E02A68B6
:100D1000920603D52A68C2F3C102D040B0FBF1F0BD
:100D200001EE900A1868B8EE612AC0F3080001EEDF
:100D3000900A1868F8EE611A40EE201A31EE810A26
:100D400022EE000AC0F34620401C00EE900AF8EEA6
:100D5000600A80EE201ABCEEC10A10EE100AF0BD47
:100D6000B6FBF1F0DCE70000104402580090D0031D
:100D70000044025840787D012C4402583444025803
:100D800000000039304402582DE9F05F0446007835
:100D9000DFF8FC8341F28839DFF8F8A3FE4DC00785
:100DA0004ED0D8F800104046C1F3C20102291AD033
:100DB0000068C0F3C200032805D1DAF8000000F093
:100DC000030002280FD06068B0F5803F12D010B148
:100DD000B0F5A02F19D0286820F48030286028684A
:100DE00020F4802009E02868800329D56068002865
:100DF00074D025E0286840F480302860606890B1A5
:100E0000FFF76CFC06464F4609E0286840F4802056
:100E10002860EFE7FFF762FC801BB8427DD82868A6
:100E20008003F7D50CE0FFF759FC06464F4604E077
:100E3000FFF754FC801BB842F0D828688003F7D431
:100E40002078D64F80075AD5D8F8001040464FF486
:100E50007C3B11F0380F13D00068C0F3C2000328A8
:100E600003D1DAF8000080070AD0E068A8B3296847
:100E700021F0190101432960FFF730FC06461DE00F
:100E80002868400702D5E0680028B1D02868E168EA
:100E900020F0190008432860FFF720FC064604E014
:100EA000FFF71CFC801B0228B8D828684007F7D53C
:100EB00007E0FFF713FC801B0228AFD82868400723
:100EC000F7D538689BFAABF220F47C312069B2FA8E
:100ED00082F290400143396011E000E0AEE0286802
:100EE00020F001002860FFF7F9FB064604E0FFF759
:100EF000F5FB801B022891D828684007F7D420789A
:100F0000C00655D5D8F8001040464FF0F84BC1F355
:100F1000C201012917D0006800E0EDE0C0F3C20073
:100F2000032805D1DAF8000000F0030001280AD0F8
:100F3000E069002828682CD040F080002860FFF786
:100F4000CDFB064616E02868C00502D5E06980287A
:100F500074D138689BFAABF220F0F841206AB2FAFB
:100F600082F290400143396022E0FFF7B7FB801B1B
:100F7000022899D82868C005F7D538689BFAABF2E3
:100F8000216AB2FA82F220F0F840914008433860BA
:100F90000EE020F080002860FFF7A0FB064604E08A
:100FA000FFF79CFB801B022887D82868C005F7D470
:100FB0002078000724D5774F60694C3700283868BF
:100FC0000FD040F001003860FFF788FB064604E0D0
:100FD000FFF784FB801B02288DD838688007F7D57F
:100FE0000EE020F001003860FFF778FB064604E0D1
:100FF000FFF774FB801B02287ED838688007F7D47F
:101000002078800623D5A069002828680FD040F4F6
:1010100080502860FFF762FB064604E0FFF75EFBA6
:10102000801B022868D828688004F7D50FE020F4D8
:1010300080502860FFF752FB064605E0D6E0FFF738
:101040004DFB801B022857D828688004F7D42078ED
:10105000400744D5524F386840F480703860FFF73D
:101060003DFB064604E0FFF739FB801B642843D8AC
:101070003868C005F7D5474FA068483701280AD01F
:1010800008B1052811D0386820F0010038603868B0
:1010900020F0040002E0386840F001003860A068E9
:1010A00088B1FFF71BFB064609E0386840F00400F2
:1010B0003860F0E7FFF712FB811B49451CD8386800
:1010C0008007F7D50BE0FFF709FB064604E0FFF7C2
:1010D00005FB811B49450FD838688007F7D4606A43
:1010E000F0B3D8F80010C1F3C20103297ED0022862
:1010F000286820F0807000E079E0286003D0FFF7D6
:10110000EDFA044687E0FFF7E9FA064604E0FFF748
:10111000E5FA801B02287BD828688001F7D4DAF82A
:10112000001040F2F3329143E26A41EA0211A26AEE
:101130001143CAF8001094F834004FF4FE02218ED7
:101140004002491EA0F5007080B2C1F308010843B7
:10115000218F491E02EA0141084394F83C1000E047
:101160005CE0491E120202EA0161084309490831A4
:1011700008600B1D19684FF6F872A06C914392FA43
:10118000A2F2B2FA82F2904001431960014809E0EC
:10119000104402582844025800440258044402589B
:1011A00000480258001D0168226C21F00C01114317
:1011B00001600168626C21F0020111430160016865
:1011C00041F480310160016841F40031016001683F
:1011D00041F480210160016841F00101016028684B
:1011E00040F080702860FFF779FA01E018E00FE026
:1011F000044604E0FFF772FA001B022808D82868AA
:101200008001F7D50AE0FFF769FA001B022802D92E
:101210000320BDE8F09F28688001F4D40020F8E79F
:101220000120F6E74FF0E0210428086903D020F000
:1012300004000861704740F00400FAE7401EB0F176
:10124000807F10B501D3012010BD4FF0E024606114
:101250000F21601700F03EFE0020A06107202061F2
:10126000002010BD7047704790F8791090F87A0010
:101270000843704770B502680446D06913689168E6
:1012800010F00F0F64D0594D03F490760D403543A4
:1012900076D0C50707D0DD0505D501251562E26FBB
:1012A00042F00102E267820708D5CA0706D0256826
:1012B00002222A62E26F42F00402E267420708D586
:1012C000CA0706D0256804222A62E26F42F00202B1
:1012D000E26702070ED503F0200201F080552A4391
:1012E00052EAC17206D0256808222A62E26F42F0F3
:1012F0000802E267E26F002A3AD0800608D503F0C0
:10130000200001F08051084302D0204600F0B2FADC
:10131000E06F000703D42068806840062AD5204685
:1013200000F09AFA2068816849061ED5816821F08C
:1013300040018160606FC0B12D490165606FFFF7AA
:1013400087F8002814D0606F016DBDE87040084731
:10135000850615D503F0200501F0805635430FD0E2
:101360002046BDE8704000F085BA2046FFF77BFFBD
:1013700070BD05E02046FFF776FF0020E067F7E745
:10138000C6024FF020050CD54E020AD5E8031062C4
:1013900084F8795084F87A502046BDE87040FFF711
:1013A00061BF06060AD503F0800601F400010E4372
:1013B00004D02046BDE8704000F0ECBC41060BD5DF
:1013C000590609D51168204621F04001116084F8C2
:1013D000795000F005F9CBE70002C9D55800C7D510
:1013E000106820F080401060C2E70000010000108B
:1013F0004518000810B5040003D094F8790010B126
:1014000007E0012010BD002084F87800204600F09D
:1014100027F8242084F879002068016821F0010170
:101420000160204600F062FA0128EBD0606B10B139
:10143000204600F075F92068416821F49041416030
:101440002068816821F02A0181602068016841F0EC
:10145000010101602046BDE8104000F0C5B9000060
:1014600010B5006886B01B49884230D11A4801681F
:1014700041F001010160006800F00100059016488C
:101480001030016841F01001016000680121134C27
:1014900000F0100005904FF4007000900220CDE99C
:1014A000010103900720694604902046FFF722F8C7
:1014B0004FF48061204600916946FFF71BF8252014
:1014C000FFF749F9032225201146FFF751F906B02D
:1014D00010BD000000100140E04402580000025816
:1014E00090F87A30202B4CD1B9B1B2B190F8783065
:1014F000012B46D0012380F878304166A0F868209F
:10150000A0F86A20FF228168B1F5805F07D07F23B1
:1015100051B1B1F1805F0CD010E00120704701693A
:1015200021B940F2FF1107E0016909BBA0F86C2066
:1015300004E00169E1B13F21A0F86C100021C1670E
:10154000222280F87A2080F8781001688A6842F0B8
:1015500001028A6001680A6892000CD50A6842F4A8
:1015600080720A600068816841F08051816006E005
:10157000A0F86C30E2E7086840F490700860002042
:10158000704702207047000030B50068114988425A
:101590000CD1114A5088010408D411464FF00003C1
:1015A0004404097806D50A2901D0538030BD40F49F
:1015B00000400DE00D2909D0084DC0F30D04401C7A
:1015C00080B2C72829555080EFD830BD40F4804004
:1015D000508030BD001001400C0000242000002489
:1015E0007047FEE7704770477047000070B5284CA1
:1015F0009CB0256825F004052560254C00260C3498
:10160000256845F440452560256805F440451B954F
:101610002568AD04FCD5012400940CAD0396240488
:10162000019402240994CDE90A410796082485E82B
:101630000D00CDE910466846FFF7A6FB88B93F20AC
:1016400013900320CDE9140640200101CDE9164096
:10165000CDE9180150201A90022113A8FFF7E6F9EE
:1016600010B101201CB070BD0A48016841F0800132
:1016700001600848F430016841F00201016000682F
:1016800000F002001B90FEF72DFF0020EAE70000AB
:101690000C48025800440258FFF726B81C4801685D
:1016A00041F4700101601B49086840F001000860C6
:1016B000184A0020103210600A68174B1A400A605E
:1016C000144A18321060121D1060121D1060114A69
:1016D00028321060121D1060121D1060121D106063
:1016E000121D1060121D1060121D1060121D10607E
:1016F0000A6822F480220A600649603108600120ED
:101700000649C1F80801C0060149803908607047E0
:1017100088ED00E0004402587FEDF6EA00800051B9
:1017200090F83410C90706D001684A68836B22F428
:1017300000321A434A6090F83410890706D50168D0
:101740004A68C36B22F480321A434A6090F834101E
:10175000490706D501684A68036C22F480221A43BF
:101760004A6090F83410090706D501684A68436C4E
:1017700022F400421A434A6090F83410C90606D594
:1017800001688A68836C22F480521A438A6090F858
:101790003410890606D501688A68C36C22F40052A9
:1017A0001A438A6090F83410490611D501684A68D6
:1017B000036D22F480121A434A60016DB1F5801F57
:1017C00006D101684A68436D22F4C0021A434A6098
:1017D00090F83410090606D501684A68806D22F435
:1017E000002202434A607047F8B500250446C567E9
:1017F000FEF774FF0746206800686FF07E4600071A
:1018000008D500223B464FF400112046009600F018
:10181000FBFA60B92068006840070AD500223B4601
:101820004FF480012046009600F0EEFA08B1032044
:10183000F8BD202084F8790084F87A00002084F82C
:101840007850F8BD10B5806B0021A0F86A10A0F8A0
:101850006210FFF708FD10BD01680A6822F490725B
:101860000A6001688A6822F001028A60202180F8FB
:101870007A10704710B5B0F86C2090F87A30016893
:10188000222B05D0088B40F008000883022010BDF1
:10189000898C8368B3F5805F01D103696BB1114016
:1018A000426E531C43661170B0F86A10491E090459
:1018B000090CA0F86A1007D015E0436E114019809A
:1018C000416E891C4166EFE701680A6822F4907254
:1018D0000A6001688A6822F001028A60202180F88B
:1018E0007A10FFF751FE002010BD00002DE9F04FE7
:1018F000044600688025FD4B0021D4F810C087B055
:10190000A6680F46D4F81C8046EA0C06D4F814C02A
:10191000A26A4CEA080C46EA0C0632430668DFF875
:10192000D0C306EA0C061643066020684268E668E3
:1019300022F44052324342602268A0699A4201D0A8
:10194000266A3043A66AB6F1005F04D1D4E90B6C75
:1019500046EA0C0630439668DFF898C306EA0C06A0
:10196000064396602068C26A666A22F00F0232431C
:10197000C262E14E2068E14AB04210D1126802F022
:101980003802182A74D005DCCAB3082A7AD0102A83
:1019900047D179E0202A7BD0282A7CD17AE0D84E22
:1019A000B04209D1126802F00702062A73D2DFE8BA
:1019B00002F053696B6D6F71D24EB04209D112685B
:1019C00002F00702062A66D2DFE802F0465C5E609B
:1019D0006264CD4EB04209D1126802F00702062AB5
:1019E00059D2DFE802F0394F51535557C74EB04234
:1019F0000BD1126802F00702062A4CD200E00EE07A
:101A0000DFE802F02A4042444648C14EB04209D1C4
:101A1000126802F03802182A38D0BBDCB4E74FF065
:101A2000010538E0BB4EB04209D1126802F007024E
:101A3000062A30D2DFE802F01026282A2C2EB64ED5
:101A4000B0420BD1126802F00702062A23D2DFE867
:101A500002F003191B1D1F2100251CE098421AD11A
:101A6000A64A121D126802F00702062A13D202E0EB
:101A70000CE007E00CE0DFE802F0030507090B0DBE
:101A8000022508E0042506E0402504E0082502E0E0
:101A9000102500E02025DFF864B2A04E9842DFF860
:101AA00080A2ABF1540B73D1102D31D006DC022D86
:101AB00009D0042D0AD0082D2FD111E0202D29D0D6
:101AC000402D2AD107E0FEF79FFE13E06846FEF79F
:101AD000B1FE01980EE003A8FEF72AFF049809E082
:101AE000DBF800105846890610D50068C0F3C10124
:101AF0002AFA01F0002811D06168894601EB410102
:101B000081420AD8B0EB093F07D808E05046F3E716
:101B10008448F1E74FF40040EEE7012733E1102D50
:101B20004FF000084ED006DC022D0FD0042D15D04A
:101B3000082D04D12DE0202D4AD0402D13D00127AF
:101B4000794AA0F54071914270D9E6E7FEF75CFE54
:101B5000626A0023414636F812200DE06846FEF71F
:101B600069FE019803E003A8FEF7E2FE0498002353
:101B7000616A36F811201946FEF7AAFB626809026D
:101B8000030241EA10615008181841EB080115E002
:101B900032E0DBF800105846890609D500680023BA
:101BA000C0F3C1012AFA01F0616A36F8112015E08C
:101BB000606A002336F8102050460FE00023FEF73D
:101BC00087FBBDE7606A002336F81020554805E022
:101BD000606A002336F810204FF400400021FEF721
:101BE00077FB0902020241EA10614FEA590010181E
:101BF0004A4641EB0801E1E7E3694FF400429342B2
:101C00004DD1082D23D005DC8DB1012D12D0042D2E
:101C100006D112E0102D35D0202D3AD0402D11D014
:101C2000012721F00F00C1F3420108435AE0FFF7FA
:101C300003F816E0FFF716F813E06846FEF7FAFD22
:101C400001980EE003A8FEF773FE049809E0DBF8A4
:101C500000105846890608D50068C0F3C1012AFA69
:101C600001F0616A36F8111010E0606A36F8101061
:101C7000BAFBF1F04100606801EB5001B1FBF0F0FC
:101C800081B2CEE7606A36F810102648B0FBF1F05A
:101C9000F0E7606A36F81000B2FBF0F0EAE7082DD2
:101CA0004AD00ADC0DB3012D43D0042D7FF44DAF93
:101CB0006846FEF7BFFD019809E0102D52D0202D97
:101CC00055D0402DF2D103A8FEF732FE0498616A88
:101CD00036F81110B0FBF1F1606801EB5001B1FB77
:101CE000F0F080B22168C8604DE01FE0000C0058A1
:101CF000F369FFCFFFF4FF11001001405444025874
:101D00000044004000480040004C004000500040AB
:101D10000014014000780040007C0040842100084D
:101D20000090D00300093D00FFFC0F00FEF784FF88
:101D3000CDE7FEF797FFCAE7DBF800205946920689
:101D40000AD50968C1F3C1022AFA02F1626A36F8BB
:101D50001220B1FBF2F20FE0616A36F81120BAFBF3
:101D6000F2F209E0616A36F811200949F1E7616A87
:101D700036F81110B2FBF1F2616802EB5102B2FBCE
:101D8000F1F189B2C16007B03846BDE8F08F0000BC
:101D900000093D0090F87910212901D002207047F8
:101DA000B0F8621021B18168B1F5805F13D014E002
:101DB00001680A68920004D58A6822F400028A60E9
:101DC00003E00A6822F080020A600068016841F0BE
:101DD000400101600CE0016961B1C16D4A1CC2653E
:101DE000026809781185B0F86210491EA0F86210E7
:101DF00000207047C16D02680988C1F30801118590
:101E0000C16D891CC165EEE72DE9F0411E461746FC
:101E100088460446069D1CE0681C1AD025B1FEF7D2
:101E20005DFC801BA84214D92068016821F4D071A0
:101E300001602068816821F001018160202084F820
:101E4000790084F87A00002084F878000320BDE847
:101E5000F0812068C16938EA010004D00020B8424E
:101E6000DAD00020F3E70120F9E7000070B50D4D4E
:101E700000240D48FFF7FEF902E0641CAC4204D8D0
:101E80000948FFF7F1F92028F7D1002402E0641C8B
:101E9000AC4206D8054901220348FFF721FB002880
:101EA000F5D170BDFFFF0100E80000240C00002404
:101EB000FEE700000FB4054B10B503A9044A0298D1
:101EC00000F028F810BC5DF814FB0000CD200008DD
:101ED000100000240907090E002804DB00F1E020AF
:101EE00080F80014704700F00F0000F1E02080F847
:101EF000141D704702E008C8121F08C1002AFAD159
:101F000070477047002001E001C1121F002AFBD179
:101F1000704700002DE9FF4F89B09B46044600251D
:101F200006E025280BD05A460B999047641C6D1C7F
:101F300020780028F5D10DB02846BDE8F08F0027A5
:101F4000B8460122474900E0074314F8013F203B0F
:101F500002FA03F00842F7D120782E2819D114F89C
:101F6000010F47F004072A280ED06FF02F022078C7
:101F7000A0F1300109290CD808EB880102EB4101DE
:101F800000EB0108641CF2E70A98641C50F8048B0B
:101F90000A9020780028CED0642808D0692806D07E
:101FA00075281ED05A460B9990476D1C58E00A9927
:101FB0004FF00A0901C90A91002802DA40422D2196
:101FC00002E0390504D52B218DF82010012103E012
:101FD000F90704D02021F7E78A4608AE0DE000217A
:101FE000FAE70A994FF00A0901C90A91F7E7494649
:101FF000FEF79FF9303106F8011D0028F7D1ADEB4F
:10200000060000F12009780701D44FF00108C84507
:1020100002DDA8EB090000E000208046002706E072
:1020200008A85A46C05D0B9990476D1C7F1C574508
:10203000F6DB04E030205A460B9990476D1CB8F14E
:102040000001A8F10108F5DC05E016F8010B5A467D
:102050000B9990476D1CB9F10001A9F10109F4DC5D
:10206000641C65E70928010010B504460420FFF749
:10207000D9F80148046010BD0800002470B50024A0
:1020800005464FF47A7603E0304600F005F8641C0C
:10209000AC42F9D370BD000070B54FF0E0250021CF
:1020A0006C69094AAB6912685043AA699A42FCD02C
:1020B00002D2A3EB020302E0A4EB0206334419446C
:1020C00013468142F1D370BD080000240349CA6958
:1020D0005206FCD5C2B20A857047000000100140CC
:1020E0000024FEF76FF9FEF707FB04230222052107
:1020F000A020FFF77BFA4FF4C870FFF7B5FF4FF44D
:10210000E13000F01BF84FF4FA75214604A0FFF708
:10211000D1FE2846FFF7B2FF641CE4B2F5E70000E9
:102120006D63756465762E74616F62616F2E636F87
:102130006D20543D25640D0A000000000B490A4A39
:1021400010B5C1E9002000208860C860086188617E
:102150000C2048610846FFF74DF9BDE810400449DE
:1021600001220248FFF7BCB900100140E80000243A
:102170000C0000240000000001020304010203041B
:1021800006070809010002000400060008000A0012
:102190000C0010002000400080000001BC2100085D
:1021A0000000002420000000F41E0008DC210008CC
:1021B00020000024480B0000041F00080090D003FA
:1021C0000090D003000000000000000000000000AC
:0C21D000010000001000000000000000F2
:040000050800029954
:00000001FF
